:020000040800F2
:100000000020002001140008651000086910000895
:1000100000000000000000000000000000000000E0
:100020000000000000000000000000006D1000084B
:1000300000000000000000007110000875100008AA
:100040005114000800000000511400085114000869
:100050005114000851140008811000088D10000888
:100060000000000099100008A910000851140008B1
:100070005114000851140008511400080000000039
:100080005114000800000000000000005114000896
:100090000000000051140008511400085114000819
:1000A000511400085114000851140008C110000830
:0800B0005114000800000000DB
:1000B80010B5064C2378002B07D1054B002B02D036
:1000C800044800E000BF0123237010BD1800002081
:1000D80000000000D05F0008044B10B5002B03D0CF
:1000E8000349044800E000BF10BDC04600000000FE
:1000F8001C000020D05F0008002243088B4274D304
:1001080003098B425FD3030A8B4244D3030B8B4210
:1001180028D3030C8B420DD3FF22090212BA030C19
:100128008B4202D31212090265D0030B8B4219D3FA
:1001380000E0090AC30B8B4201D3CB03C01A52411A
:10014800830B8B4201D38B03C01A5241430B8B4262
:1001580001D34B03C01A5241030B8B4201D30B034B
:10016800C01A5241C30A8B4201D3CB02C01A524172
:10017800830A8B4201D38B02C01A5241430A8B4235
:1001880001D34B02C01A5241030A8B4201D30B021E
:10019800C01A5241CDD2C3098B4201D3CB01C01A38
:1001A800524183098B4201D38B01C01A5241430942
:1001B8008B4201D34B01C01A524103098B4201D330
:1001C8000B01C01A5241C3088B4201D3CB00C01A9D
:1001D800524183088B4201D38B00C01A5241430815
:1001E8008B4201D34B00C01A5241411A00D201463A
:1001F800524110467047FFE701B5002000F0F0F8C3
:1002080002BDC0460029F7D076E7704703460B4386
:100218007FD4002243088B4274D303098B425FD3F7
:10022800030A8B4244D3030B8B4228D3030C8B4223
:100238000DD3FF22090212BA030C8B4202D3121209
:10024800090265D0030B8B4219D300E0090AC30BDE
:100258008B4201D3CB03C01A5241830B8B4201D38B
:100268008B03C01A5241430B8B4201D34B03C01A74
:100278005241030B8B4201D30B03C01A5241C30AEC
:100288008B4201D3CB02C01A5241830A8B4201D35D
:100298008B02C01A5241430A8B4201D34B02C01A47
:1002A8005241030A8B4201D30B02C01A5241CDD2EC
:1002B800C3098B4201D3CB01C01A524183098B4237
:1002C80001D38B01C01A524143098B4201D34B0120
:1002D800C01A524103098B4201D30B01C01A524183
:1002E800C3088B4201D3CB00C01A524183088B420A
:1002F80001D38B00C01A524143088B4201D34B00F3
:10030800C01A5241411A00D2014652411046704764
:100318005DE0CA0F00D04942031000D34042534069
:1003280000229C4603098B422DD3030A8B4212D329
:10033800FC22890112BA030A8B420CD3890192115B
:100348008B4208D3890192118B4204D389013AD098
:10035800921100E08909C3098B4201D3CB01C01A6D
:10036800524183098B4201D38B01C01A5241430980
:100378008B4201D34B01C01A524103098B4201D36E
:100388000B01C01A5241C3088B4201D3CB00C01ADB
:10039800524183088B4201D38B00C01A5241D9D2F3
:1003A80043088B4201D34B00C01A5241411A00D274
:1003B8000146634652415B10104601D34042002B70
:1003C80000D54942704763465B1000D3404201B5EF
:1003D800002000F005F802BD0029F8D016E77047A4
:1003E8007047C0469E2110B5C905041C00F078FB73
:1003F800002803D1201C00F0E1FA10BD9E21201C2A
:10040800C90500F02DF900F0D9FA80231B069C4697
:100418006044F2E7F0B54F464646D64644024500EA
:10042800C0B5640A0F1C2D0EC60F002D00D18DE03B
:10043800FF2D00D192E00023802099469A46E400DF
:10044800C00404437F3D7802430A98467B001B0E94
:10045800FF0F002B00D170E0FF2B00D186E0424651
:10046800D00080227F3BED180023D204024390463F
:100478009C4631004B467940681C0F2B1CD8764AA5
:100488009B00D3589F4639004446E2465346022B08
:100498000FD0032B00D1D7E0012B37D10020002447
:1004A800C0052043C9070843E0BCBA46B146A84680
:1004B800F0BDFF200024F3E7260C2404220C444658
:1004C8002404240C434627001B0C574374435A4307
:1004D8005E4312193B0C9B189C4203D9802252029E
:1004E800944666443F041A043F0CD2199401671ECF
:1004F800BC411B0C920E9B1914439B011C431B010E
:1005080000D49BE0012362081C40144302007F32A0
:10051800002A64DD630704D00F232340042B00D096
:100528000434230103D502004C4B80321C40FE2AC0
:10053800BFDCA401640AD0B2B2E74346002B3DD128
:100548004A4601331A4391469C4692E7002C29D12A
:1005580004239946033B00259A4674E7002C1BD1D7
:1005680008239946063BFF259A466CE74346FF3524
:10057800002B0BD102234A461A4391469C4678E742
:1005880053463100022B00D083E792E703234A4603
:100598001A4391469C466CE70C239946093BFF2574
:1005A8009A4650E7200000F0A5FA7625431F9C40A4
:1005B80000236D4299469A462D1A44E7404600F0BA
:1005C80099FA4246431F9A4000232D1A90469C46AA
:1005D800763D4EE780240021FF20E40360E70123F5
:1005E8009B1A1B2B00DD59E722009E30DA4084401D
:1005F8001300621E94411C43630704D00F23234059
:10060800042B00D0043463011AD50120002447E7E5
:100618008020C003044209D04346034206D1444621
:10062800044364023900FF20640A39E78020C003CC
:10063800044364023100FF20640A31E7280065E7BB
:10064800A4010020640A2BE78020C003044364024D
:10065800FF20640A24E7C046E85F0008FFFFFFF7B1
:10066800F8B5CE46474643025B0A4E02DA00944686
:10067800720A914645004A0080B52D0E1F00C40F2E
:10068800120EC90FB609FF2A5BD0012041408C42E7
:1006980039D0A81A00285ADD002A6AD0FF2D00D1C7
:1006A800D9E08022D20416431B2800DCE9E00120AF
:1006B8006346181A430100D4B4E080018709380062
:1006C80000F018FA05388740854200DCCCE02D1A86
:1006D800B5483840430704D00F230340042B00D00B
:1006E8000430430100D4A0E06A1CFE2D00D18DE047
:1006F8008001470AD2B2D0053843E4072043C0BC82
:10070800B946B046F8BDA81A8046002845DD002A3B
:1007180070D0FF2D00D19EE08023DB041E434346AA
:100728001B2B00DCD2E00120604443017AD501355F
:10073800FF2D6BD001239D4A034040081040184309
:10074800C8E7002E20D08C4223D02800FF3800288C
:1007580039D0571B002D00D09DE06346002B00D1F7
:10076800DBE07B1E012F00D10DE1FF2F71D01F00B0
:1007780098E0002E00D1A7E0421E012800D1E6E053
:10078800FF2868D010008FE701204140A14200D027
:100798007FE7FF2040428046A8444046002838D0E2
:1007A800511B002D00D1AEE0FF2A00D1DFE08023ED
:1007B8006046DB04184384461B2900DCD9E001208D
:1007C80015008019B1E7FE206A1C104271D1002D76
:1007D80000D0A6E06346002B00D1D9E00022002E0D
:1007E80000D188E7981B430100D4E1E063460C0080
:1007F800F01A6FE7002E00D1B7E00200013A012895
:1008080000D19CE0FF2826D0904688E7FF220027E9
:1008180071E7FE206A1C104264D0FF2AF6D015004A
:1008280066447008430700D056E7C308FF2D12D06E
:100838005B025F0AEAB25EE76246002A00D196E0F0
:10084800002E08D08022D203134204D0484610421A
:1008580001D10C004B46002BD8D08027FF031F4343
:100868007F02FF227F0A46E720233A00451B380013
:100878000135EA405D1BA840431E984100251043FE
:1008880028E720231B1A32009E40C2403000431E36
:10089800984110430CE7FF2ADBD080236046DB0435
:1008A800184384461B2F56DD01200C001500301A12
:1008B80000E763469F1B7B013DD4002F00D0FEE676
:1008C80000240022002716E70500AFE73200434660
:1008D8004146DA4020235B1A9E403000431E98416F
:1008E800104321E7002DA7D16346002B59D00022E1
:1008F800002E00D1FFE630006044430192D52A4B18
:10090800013518408EE76346002B47D04B1E01295E
:1009180015D0FF292BD019004EE70C004B463D009F
:1009280084E76246002A8BD1002E92D180270024CA
:10093800FF22FF03DFE663460C00F71ABFE630002C
:1009480060440125430100D46CE70225F2E66346C2
:100958000125981BAEE6202364466046FC40DF1B59
:10096800B840431E984120439FE705005EE74B4689
:1009780071E7202365466046CD40591A8840431EDA
:10098800984128431CE763460C000125F01A91E6BC
:10099800002E95D00C004F460022ACE64B460D00C9
:1009A80044E74F460022A6E6FFFFFFFBFFFFFF7D5F
:1009B800002800D036E7002400279CE641024200C8
:1009C800C30F490A0020120E7E2A03DD9D2A02DD8C
:1009D800094A98187047802000040143952A07DCCB
:1009E8009620821AD1404842002BF3D10800F1E743
:1009F800963A9140F7E7C046FFFFFF7F70B5051EA6
:100A08000ED000F077F89E2304001B1A962B0CDCFE
:100A1800082801DD083CA5406D026D0AD8B201E046
:100A280000200025C005284370BD992B09DD020070
:100A380029001B3291404A1E91410522121AD540C5
:100A48000D43052C12DC29000C4E31406A0709D0F1
:100A58000F202840042805D004314A0102D59F23DD
:100A680031401B1B89014D0AD8B2DBE7621F954054
:100A78002900024E31406A07F4D0E9E7FFFFFFFB87
:100A8800844608006146FFE71FB500F0BDF800285E
:100A980001D40021C8421FBD10B500F049F84042FA
:100AA800013010BD10B500F0AFF8002801DB0020C0
:100AB80010BD012010BDC04610B500F0A5F80028F3
:100AC80001DD002010BD012010BDC04610B500F0AA
:100AD80055F8002801DC002010BD012010BDC046DB
:100AE80010B500F04BF8002801DA002010BD0120F5
:100AF80010BDC0461C2101231B04984201D3000CE1
:100B080010391B0A984201D3000A08391B09984278
:100B180001D30009043902A2105C40187047C0468E
:100B280004030202010101010000000000000000AE
:100B380070B5420045024E024C00C30F6D0A0120F9
:100B4800120E760A240EC90FFF2A06D0FF2C03D0F6
:100B5800A24201D1B54206D070BD002DFCD1FF2CB8
:100B6800FAD1002EF8D18B4206D00120002AF3D109
:100B78002800431E9841EFE70020EDE770B54200DA
:100B880045024E024C00C30F6D0A120E760A240E5F
:100B9800C80FFF2A1BD0FF2C0ED0002A1BD1002C17
:100BA80001D1002E1CD0002D0CD083421CD0022174
:100BB800581E0840013870BD002E22D1002AF4D1F9
:100BC800002DF2D10028F6D101204042F3E7002D94
:100BD80017D1FF2CF0D0002CE7D1002EE5D1E6E7A5
:100BE8000020002DE7D0E2E7A24205DCEADBB542AF
:100BF80002D8E7D30020DEE74342584140000138DD
:100C0800D9E702204042D6E770B5420045024E02BD
:100C18004C00C30F6D0A120E760A240EC80FFF2A65
:100C28000BD0FF2C0DD0002A1FD1002C16D1002E7E
:100C380014D10020002D10D009E0002D0CD1FF2C7C
:100C480013D1002E08D1002A08D0834212D00221E5
:100C5800581E0840013800E0022070BD002DF4D174
:100C68000028FAD101204042F7E7002CEDD1002EF0
:100C7800EBD1ECE7A24205DCF2DBB54202D8EFD3B8
:100C88000020EAE74342584140000138E5E7C04602
:100C980010B584B00C220021684605F08CF980223A
:100CA800194C120622610422012162610022174BAD
:100CB800A17623608023E1612B3100206254072153
:100CC8001B0363600023206361633C2120002383AE
:100CD800A360E3606362A3626254E36400F002FC11
:100CE80000280BD101230A4A69462000009201938B
:100CF80000F074FD002804D104B010BD00F094F990
:100D0800F0E700F091F9F7E73800002000240140EF
:100D18000200000470B504008EB01422002102A85D
:100D280005F049F91822002108A805F044F9274BD5
:100D380022689A4201D00EB070BD8023DB0108936F
:100D4800802308A81B060C9302F0D8F9002837D195
:100D580080201F4B4003196C0026014319641A6C4C
:100D680002400092009A0122596BA0201143596356
:100D78005B6BC0051A400192019B0222032302A962
:100D880002920393049601F0F7FB124D124B2800D0
:100D98002B6005236B607B332B6180336B61802371
:100DA800DB00AB612023EB6180235B01AE60EE606A
:100DB8002B6201F039F8002805D12565AC62BAE745
:100DC80000F032F9C4E700F02FF9F6E700240140FB
:100DD800001002409C0000200800024001230E4A37
:100DE80000B5916B83B019439163926B0221134054
:100DF800019300220920019B00F0AEFF092000F0BA
:100E0800DDFF002202210A2000F0A6FF0A2000F0E0
:100E1800D5FF03B000BDC04600100240F0B5CE4675
:100E280000B588B01422002102A805F0C4F80222F7
:100E3800424BA024596BE40511435963596B2000B8
:100E48000A400092009A0122596B3D4D11435963A3
:100E58005B6B3C491A4001920122019B01F02CFD79
:100E680020000022202101F027FD28000122012175
:100E780001F022FD042201230292039300220023A1
:100E8800200002A90492059301F076FBC4230822EE
:100E98009B03029203930023200002A9994600268F
:100EA8000227049301F068FB20220123200002A9F5
:100EB800029203930496059701F05EFB40220023FB
:100EC800029203934B46200002A9049301F054FBBD
:100ED800882380225B03029203934B46200002A9D9
:100EE800049301F049FB012201230292039300229B
:100EF8000023280002A90492059301F03DFBC022BB
:100F080011232000520102A9029203930496059727
:100F180001F032FB00220221062000F01DFF06200E
:100F280000F04CFF00220221072000F015FF0720E7
:100F380000F044FF08B080BCB946F0BD0010024084
:100F480000040050041800000848094B10B503605D
:100F580003234360074BC360074B836001F0D4FC55
:100F6800002800D110BD00F05FF8FBE7F800002072
:100F780000300040FF0F0000B80B000000B593B030
:100F88003422002105A805F016F810220021684631
:100F980005F011F88020800001F0F4FC0A23059385
:100FA800F6330893002309930E9308330F93802395
:100FB80040229B02109380230A923F3A0B929B0592
:100FC800013205A80C920D92119301F00BFD002837
:100FD80001D072B6FEE70722022300920193002295
:100FE8000023022168460292039301F0ABFF002818
:100FF80001D072B6FEE713B000BDC04610B500F0D0
:101008004BFAFFF7BBFF04F05BFEFFF707FFFFF7A4
:10101800E5FEFFF73DFE00F085F800F0F9F8FFF770
:1010280093FF04F0BBFCFEE772B6FEE701220A4B11
:1010380082B0196C11431964196C0A40802100921E
:10104800009ADA6B49050A43DA63DB6B0B400193BC
:10105800019B02B07047C04600100240FEE7C04640
:10106800FEE7C0467047C0467047C04610B500F05E
:1010780027FA04F069FE10BD10B5082001F02AFC1B
:1010880010BDC04610B5802001F024FC10BDC0463C
:1010980010B5024801F08CF810BDC0469C00002035
:1010A80010B5034801F084F8024801F081F810BD3A
:1010B80054010020B001002070B5144C200002F04B
:1010C8005DFE200002F00CFD10222368D9690A4257
:1010D80004D01A620E4B1A78002A06D00D4D29004A
:1010E8008022200002F07EFC70BD0B4A094D126878
:1010F8000A48516880225242521AD2B21A701A789B
:101108002900D2B204F04EFFE9E7C0460C020020E5
:1011180094060020F004002054010020140600204A
:101128007047C04610B590B01C22002108A804F0F2
:1011380042FF284C284B294A23600223636000237E
:101148002000A360E2602361A36102F095F8002803
:101158001ED1200002F032F9002820D1FA236022A3
:101168009B000892099300230022200008A90A93F3
:101178000C9302F023FA002814D11422002102A8AB
:1011880004F019FF144B22689A420ED010B010BD1B
:10119800FFF74AFF200002F011F90028DED0FFF720
:1011A80043FFDBE7FFF740FFE7E701230C4AA020F6
:1011B800516BC00519435163526B02A91340019347
:1011C8001022019B0223029203930423069301F049
:1011D800D3F9DBE70801002000200040E703000006
:1011E80000100240084B026882B09A4201D002B057
:1011F80070478020054A0002116C01431164136C8A
:1012080003400193019BF2E70020004000100240D8
:1012180010B5214B214C0C22236096239B0163605F
:1012280000232000A360E36023616261A361E3619E
:1012380023626362A36203F0C9F8002811D1002178
:10124800200003F0FFF9002813D10021200003F04B
:1012580049FA002815D1200003F0D8F9002817D141
:1012680010BDFFF7E1FE0021200003F0EBF9002894
:10127800EBD0FFF7D9FE0021200003F033FA002855
:10128800E9D0FFF7D1FE200003F0C0F90028E7D02D
:10129800FFF7CAFEE4E7C046003801400C02002010
:1012A80070B504008EB01422002102A804F083FE59
:1012B8001822002108A804F07EFE364B22689A42C4
:1012C80001D00EB070BD012308A8089301F016FFE5
:1012D800002856D18020304BC001196C00260143EC
:1012E80019641A6C02400092009A0222596B2B482A
:1012F800114359635B6B02A91A400192019BC022FA
:101308000223029203930023002206960492059377
:1013180001F032F9224D234B28002B6032236B60F9
:101328004E332B6180235B01AE60EE606E61AE616F
:10133800EE612B6200F078FD002828D180221A4B3C
:10134800A550AC62194D2B6033236B60233BAB6017
:101358000023EB606B61AB61EB61802328005B01CC
:101368002A612B6200F060FD00280DD100220121C6
:101378001B20E567AC6200F0EFFC1B2000F01EFDAF
:101388009FE7FFF751FEA5E7FFF74EFEEEE7FFF7F1
:101398004BFED3E700380140001002400004005023
:1013A800540100201C00024030000240B00100201F
:1013B8000D4B026810B504009A4200D010BD0B4ACC
:1013C8000B49136C0B480B401364C02101F0E2F980
:1013D8008023E05800F0A0FDE06F00F09DFD1B2089
:1013E80000F0F8FCEAE7C04600380140001002406F
:1013F800FFBFFFFF000400500D488546FFF790FE31
:101408000C480D490D4A002302E0D458C450043357
:10141800C4188C42F9D30A4A0A4C002301E013602D
:101428000432A242FBD304F099FDFFF7E7FDFEE783
:10143800002000200000002018000020246100087F
:101448001800002008070020FEE7000010B50F4B29
:1014580004001978002901D1012010BDFA2080006C
:10146800FEF74AFE0A4B01001868FEF745FE00F039
:10147800C1FC0028F0D1032CEED80138002221004D
:1014880000F06AFC034B00201C60E6E70400002023
:1014980000000020080000208023084A5B00116833
:1014A80010B50B4303201360FFF7D0FF041E02D0D2
:1014B8000124200010BDFFF7B9FDFAE70020024023
:1014C800034A044B11681B785B1813607047C046C9
:1014D800A002002004000020014B18687047C04695
:1014E800A0020020F0B5C646002300B582B0041E55
:1014F800019300D1DBE0856D002D00D1ABE08023A6
:1015080025685B05AA681A4215D1AA687E490A406F
:101518001343AB607D4B7E491868FEF7EDFD013043
:1015280040000190019B002B05D0019B013B0193DA
:10153800019B002BF9D1AB680020DB0000D47DE0D3
:10154800AB685B0709D5A36D10220120A36D134377
:10155800A36502B080BCB846F0BDA36DDB06F3D42A
:10156800A36D6C4A13400632FF321343A365AB6880
:10157800DB0776D4A67E637E7703BC46217E276B85
:10158800DB039846A2688903002F01D080277F01DA
:10159800E3681A4343460A431A43634621691A43D8
:1015A800002900DA9FE080239B039C462C23E35C00
:1015B8005B0013433B43624620271343E25D012A45
:1015C80000D194E0626A002A05D0E0267600324015
:1015D800A66A32431343EA684F4E676832401343A2
:1015E800BE0FE26CEB60B30798461A433C23E35CFA
:1015F8009C46012B09D1236C666C33431343A26CC0
:1016080013434246134362461A432B69434E334001
:10161800134380222B617B005B08D205934221D0C3
:1016280080231B069F421DD03D4A3E4E136833401F
:10163800F026B60337401F43176013E01022A36D4E
:1016480001201343A365E36D0F3A1343E365AB68C9
:101658005B0782D577E7FFF75DFB5423E565E55423
:101668004DE72169072270276B69666B9343334303
:101678006B616A69A36BBA431B0113436B61002951
:1016880017D11023AA6A5B421343AB6207236A6926
:1016980013409E421ED01222A36D01209343023AAA
:1016A8001343A365E36D0F3A1343E36551E7012044
:1016B8004FE780239B039942E8D11C22AB6AE36978
:1016C800013B9B001A4010235B429340226E134358
:1016D800AB62DBE700230322E365A36D9343023A81
:1016E8001343A36535E74B005B089C465EE7002E75
:1016F80003D180225202134364E7A66D3743A765DE
:10170800E66D3243E2655DE7E8FFFF6F0000002009
:10171800400D0300FDFEFFFF0102FEFF02FCFF1F5C
:1017280008270140FFFFC3FF7047C0467047C04607
:1017380010B5806AFFF7FAFF10BDC0467047C04673
:101748004022806A10B5836D13438365C36D3C3AAC
:101758001343C365FFF7F2FF10BDC04650210300D5
:10176800806A10B5826D11420DD18023826D9B0075
:101778001343C022836503681201D96811420AD055
:10178800FFF7D2FF10BD826DD20616D4026D180085
:10179800526B9047F6E7827E002AF1D11A68120749
:1017A800EED59A6852070BD52022836D13438365C3
:1017B800C36D1F3A1343C365E2E7FFF7BFFFE1E7D5
:1017C8000C215A688A435A60836D034A13400432D5
:1017D800FF3213438365D3E7FEFEFFFFF0B54546AE
:1017E800DE4657464E460023E0B585B00393543392
:1017F800C25C04000569012A00D191E0012004229D
:10180800E05423689E6832420DD0A36D1C32134306
:10181800A36554230022E25405B0F0BCBB46B2468F
:10182800A946A046F0BD4E689543022E5CD080279D
:101838003F06BD4251D0256E0F27AA461F25AC464C
:101848003540AF40A946FD4300955546BD43A846DF
:101858000D6801976F036CD16046AA0E1040020014
:10186800484682404046104380464246B6082266B3
:10187800E2690136964208D84E46AA00120FB240D5
:10188800986A009E304002439A6228028A680100E2
:101898005E69024066488E43024032435A61002D19
:1018A80001DB0020B5E7E0216248634A0368490488
:1018B8001940954251D0614A954245D0604A9542B7
:1018C800EFD18025ED032B42EBD102685D4B1A4026
:1018D8000A431543056000209BE70D68986A6A0370
:1018E800520B02439A62D0E780221206954219D021
:1018F8000A68002AD5DA4F494F480B68824229D036
:101908004E4882424CD04E488242CAD1C0200A6812
:10191800400403404B480240134300200B6078E723
:10192800022079E70A68996A5003400B814399625B
:10193800DFE7284299D102272F422DD04A4690400E
:1019480042460243904690E780256D042B42BCD066
:1019580000205EE7A0200A68DAE780252D042B42E4
:101968009FD10268374B1A400A43374B154305602D
:1019780018683649FEF7C0FB013043001B189B006E
:101988000393039B002B8CD0039B013B0393039B86
:10199800002BF9D100203CE72A4205D03A005FE746
:1019A800C0200A680004B4E72A0701D5032257E7D4
:1019B800EA0601D5042253E7AA0601D505224FE716
:1019C8006A0601D506224BE72A0601D5072247E712
:1019D800EA0501D5082243E7AA0501D509223FE710
:1019E8006A0501D50A223BE72A0501D50B2237E70C
:1019F800EA0401D50C2233E7AA0401D50D222FE70A
:101A08006A0401D50E222BE72A0404D55246019810
:101A18000243904629E7EA0301D5102220E7AA03EA
:101A280001D511221CE76A0300D41EE7122217E72A
:101A380000FFFF0708270140001000B0004000B871
:101A4800002000B4FFFF3FFE00000020400D03000F
:101A5800036870B59A680400520716D59A68920709
:101A680015D5FFF739FD236806009B685B070CD581
:101A78000425FFF731FD2368801B022802D99A68E4
:101A8800154212D19B681D42F3D1002070BD9A689F
:101A98000B490A4010210A439A60FFF71DFD23688D
:101AA80006009B685B07E3D4EFE71022A36D0120D3
:101AB8001343A365E36D0F3A1343E365E6E7C046B6
:101AC800E8FFFF7F00230122F0B583B0019303688C
:101AD800040099680A421FD19868284908421ED113
:101AE8009968274801400A439A60264B1B681B02E5
:101AF8000FD5254B25491868FEF7FEFA01300190ED
:101B0800019B002B05D0019B013B0193019B002BFE
:101B1800F9D1637E012B0BD1002003B0F0BD102159
:101B2800A36D01200B43A365E36D1A43E265F4E757
:101B3800FFF7D2FC236806001A68D207ECD4012507
:101B48000F4F9A68154203D19A683A402A439A601F
:101B5800FFF7C2FC2368801B022802D91A681542C5
:101B680003D01A681542ECD0D6E71022A36D0120E5
:101B78001343A365E36D1D43E565CEE717000080B9
:101B8800E8FFFF7F0827014000000020400D030008
:101B9800F0B5C64605680400AE68884617000220FE
:101BA80000B5730714D45422A35C012B10D0012371
:101BB800A354EA68134206D1AA68134231D101221C
:101BC800EB681343EB602000FFF77CFF002802D08E
:101BD80080BCB846F0BDA36D154A256D1A40802318
:101BE8005B001343A365134BE065EB62124B1022B5
:101BF8002B63124B21686B631C230B603833E05452
:101C08004B68280013434B6042463B00403100F0CC
:101C1800EBF922680A4993680B4004210B4393604F
:101C2800D6E7AB68064A13401843A860C7E7C04622
:101C3800FEF0FFFF6517000839170008491700086C
:101C4800E8FFFF7F0222F8B50368040099680A429A
:101C580002D000209B68F8BD01219868014228D075
:101C6800052798680740012F08D01022A36D01208E
:101C78001343A365E36D1943E165ECE799681248DE
:101C8800012501400A439A6003221A60FFF724FCE9
:101C9800236806009B681F420BD0FFF71DFC2368D2
:101CA800801B022802D99A68154204D19B681D42FC
:101CB800F3D10020CFE71022A36D01201343A365C1
:101CC800E36D1D43E565C6E7E8FFFF7F542370B564
:101CD800C25C0400012A25D00122C254FFF7B8FED5
:101CE800051E1AD12523206DC35C022B1CD01021A0
:101CF8002268200053688B435360FFF7A3FF051E3B
:101D080006D1A36D134A13400432FF321343A3656F
:101D180001212268D3688B43D36054230022E25404
:101D2800280070BD0225FBE700F0C6F9051EDED0CD
:101D380040221021A36D200013432268A365536835
:101D48008B435360FFF77EFF01212268D3688B43E2
:101D5800D360E2E7FEFEFFFF70B5002814DB154BE9
:101D680003229C46FF23840810401A00C026C000A6
:101D7800890182400B408340A4006444B600A55901
:101D880095432B43A35170BD0B4A0F23944603225E
:101D980003401040FC321500C000890185400A400C
:101DA8008240083B9B089B006344DC69AC432243A8
:101DB800DA61E8E700E100E000ED00E0002805DB7B
:101DC8001F2318401E3B8340014A13607047C046DA
:101DD80000E100E000280ADB1F2318401E3B834077
:101DE800802203498B50BFF34F8FBFF36F8F70472B
:101DF80000E100E08022431E5204012093420ED2EB
:101E0800C021074A07485360036A09061B021B0AD8
:101E18000B4303620023002093600733136070476D
:101E280010E000E000ED00E0F0B5C646040000B5A3
:101E3800002862D00568324B1421E818FEF75CF9D7
:101E48008300236402222523E2542B682D4AA668C6
:101E580013402B60E368216933430B4361692A68A7
:101E68000B43A1690B43E1690B43216A0B431343FD
:101E78002B60254B14219C4660448700FF20234B90
:101E88002840A364676408389846FEF735F91F238D
:101E980001220340100098408023E064DB019E4249
:101EA80021D03F23454661680B4001393B6068609B
:101EB80003291DD803201649164D5918013B034024
:101EC8009A400023890021656565A2650B606A60F8
:101ED8000023252201210020E363A154013AA354E1
:101EE80080BCB846F0BD002363603B604346586041
:101EF800002323656365A365EAE70120F0E7C04690
:101F0800F8FFFDBF0F80FFFF00820010800802402D
:101F18003F82001040090240F8B5CE46474604000B
:101F280080B5002851D003680126984642461B68B0
:101F38002748B343136014214044FEF7DDF8002717
:101F480043468500234925641F604B681C229C4634
:101F580033002A409340624613434B601E4B1421C2
:101F68009C461E4B604485009946A364FF20434667
:101F7800184065640838FEF7BFF81F233200034095
:101F88009A401300E2644A462F60536063685A1E01
:101F9800032A11D900232522002023656365A36540
:101FA800E36223636363A363E363A354013AA35423
:101FB800C0BCB946B046F8BD094996408C46634452
:101FC8009B001F60074B5E60E4E70120F0E7C04616
:101FD800F8FFFDBF000002400082001080080240A8
:101FE8003F82001040090240F0B5C646242400B5DF
:101FF800055D012D4FD0012525260555855DEFB2DC
:10200800012D07D08023C36300230355012080BC22
:10201800B846F0BD223C84550024C4630468C66CED
:102028002568BD432560856C6E60066D002E02D064
:10203800456D876D6F601C271E4DAC466D68A846C0
:10204800056C2F400125BD4047463D4367467D60EE
:1020580063608368102B20D0A160E260036B002BC3
:102068001ED00E22236813432360436C1A68D203E0
:1020780004D58022196852000A431A60002E04D041
:10208800802332685B0013433360012223680020F9
:1020980013432360BBE70220B9E7A260E160DDE7F4
:1020A8000422236893432360236806321343236082
:1020B800DBE7C0460000024070B5002834D0252375
:1020C800C35C022B29D10E210268184C1368066CD8
:1020D8008B43416C13600B6823400B60012311682C
:1020E800994311601C223240934011494D682B439B
:1020F8004B60C26C836C5A60036D002B05D01A6864
:1021080014401C60826D436D5A6025230122C2541D
:102118000022013BC254002070BD04230022C36387
:102128002033C2540120F7E70120F5E7FFFEFFFF47
:1021380000000240252370B5C35C022B03D00423A2
:10214800C363012070BD0E210268174C1368066C2A
:102158008B4313600123116899431160416C0A682D
:1021680022400A601C223240934010494D682B439C
:102178004B60C26C836C5A60036D002B05D01A68E3
:1021880022401A60436D826D5A6025230122C25491
:102198000022013BC254836B002B02D098470020D9
:1021A800D0E70020CEE7C046FFFEFFFF0000024058
:1021B8002C4B70B51A6804251C23046C0168234055
:1021C8002C009C400E68224210D035420ED00B687D
:1021D8009B0602D40B68AB430B60224B5A6814432E
:1021E8005C60036B002B00D0984770BD02252C0063
:1021F8009C40224217D0354215D00B689B0606D466
:102208000A220B6893430B602523093AC254154BE5
:102218005A6814435C6000222423C254C36A002B0A
:10222800E3D09847E1E7082425009D402A42DCD006
:102238003442DAD00A680634A2430A600122150043
:102248009D402B0007494C6823434B602523C263FC
:10225800C2540022013BC254436B002BC5D098479F
:10226800C3E7C046000002402523C05CC0B27047E7
:10227800C06B7047F0B54546DE464E465746E0B55A
:102288009B465C4B83B098461B7881460D000192B3
:10229800012B2BD042460123137000235360FFF714
:1022A8001BF9FA2380249B00534FC618640203E0ED
:1022B800FFF712F9864217D93B692342F8D13A69E8
:1022C8004E4B10004E49184039611A4210D043460F
:1022D8005860012000234246137003B0F0BCBB468F
:1022E800B246A946A046F0BD0320F3E70220F4E772
:1022F800FFF7F2F8FA239B00C7188023DB029A46FF
:102308003D4E03E0FFF7E8F88742EDD952463369BE
:102318001342F7D14B46012B45D0524673691A43F5
:102328007261EFF3108072B6019A13002B435B07BA
:1023380056D1131DAB4253D01400511CFF31AD1AB6
:102348002B192668676808341E605F608C42F7D1D5
:102358008022294952020B691342FCD180F310886C
:10236800FFF7BAF8FA2380269B00234DC41876029B
:1023780003E0FFF7B1F8844213D92B693342F8D14F
:102388002A691E4B10001E49184029611A4215D0AF
:102398004346586001204946174A53698B435361A5
:1023A80098E70320F7E74A46736913437361019B73
:1023B8002B60BFF36F8F5B466B60D1E7FFF78CF83C
:1023C800FA2380259B000C4EC418ED0203E0FFF7AA
:1023D80083F88442E5D933692B42F8D10020DAE743
:1023E800019C631CFF332D1B22682A510434A3422D
:1023F800FAD1ADE7A402002000200240FA830000D1
:10240800FB830000054B00205A69002A05DA044ABC
:102418009A60044A9A605869C00F704700200240C9
:1024280023016745AB89EFCD8022044B1206596919
:102438000A435A615869C043C00F704700200240E0
:10244800F8B507008026FFF747F8144DC41976023F
:1024580003E0FFF741F8A0420ED22B693342F8D1CE
:102468002A690F4B10000F49184029611A4205D0FC
:102478000D4B5860012000E00320F8BDFFF72CF851
:102488008025064E3F18ED0203E0FFF725F8874246
:10249800F2D933692B42F8D10020EEE70020024040
:1024A800FA830000FB830000A4020020F0B54F4629
:1024B8004646D6462B4B050098461B788946C0B53C
:1024C800012B42D042460123FA20137000238000DA
:1024D8005360FFF7B5FF071E2ED104236B602B68EE
:1024E800042B34D001234A465B421360AC68EB6886
:1024F800E3189C421BD21C4B1C4E9A4606E0EA6825
:10250800AB68944601346344A34210D95146FA207B
:102518007269E3000A401343154A8000134373614C
:10252800FFF78EFF0028EAD04B4607001C60022107
:102538000E4A53698B435361002342461370380097
:10254800E0BCBA46B146A846F0BD0227F7E7FA2034
:10255800064A084B516980000B435361FFF770FF2F
:102568000700E9E7A402002007E0FFFF002002407F
:102578000200010004000100F0B5DE4657464E4651
:102588004546E0B50C688C460022002383B0002C39
:1025980000D180E07B498B466146019101262100EC
:1025A8009E4031408A4634426FD0019D69680325B8
:1025B8000D40AC46013D012D00D873E06546032D62
:1025C80000D0B7E066469640F54300950768009D41
:1025D8003D4035430560C025AD02294255D0694EBE
:1025E8000327B4469D081F40FF00AD006544BC4664
:1025F8002E6E0F27B1466646B7403E004F46B7439A
:10260800B946A027FF05B84212D05F4FB84200D1A3
:10261800A8E05E4FB84200D1ACE05D4FB84200D1AF
:1026280099E066460527B7403E004F463743B9460E
:102638004E462E66564680275D46F6437F03B046D3
:102648002D68394200D083E035405F463D607D68A3
:102658008027BF03394200D077E0464635405F46C1
:102668007D6084257D598E036CD446463540842789
:10267800BC465F466646BD5180257D59C9035ED478
:1026880046462E40802559464E5121000133D940F7
:102698000232002982D103B0F0BCBB46B246A9463B
:1026A800A046F0BD8568A84603259540EF430097EE
:1026B8004746AF43019DB946EF689740B8464F4635
:1026C80045462F43876045682F000125B7430E090B
:1026D8002E409E403E434660C668009D2E40B04650
:1026E800019D4746AE6896403E43C66067466646CB
:1026F8009640022F00D069E7DD08AD00AC4684445F
:1027080065462D6AA94607252F001F40BD000F27E3
:10271800A846AF404D46BD434746A946019D2D6991
:10272800BD40A8464D4647463D43A94665464F46E7
:102738002F624BE703259540ED430095CCE75646BD
:102748002E439FE75646354391E75646354386E77D
:102758005646354379E767460326BE404F4637431A
:10276800B94665E766460127B7403E004F463743FE
:10277800B9465DE767460226BE404F463743B9462D
:1027880056E7C046001802400004005000080050F8
:10279800000C0050F0B5DE4657464E464546E0B5BB
:1027A800002383B0002965D0012291460232934666
:1027B8003A4A944644E03A4CA04262D0394CA0428E
:1027C80063D0394CA04264D00524AC402500AE4209
:1027D80014D18024654666462D59BD4335510434CD
:1027E8003559BD43355144467568BD4375603568F4
:1027F800BD433560019E356EA54335665E465D0076
:10280800AE400468350034430460DC08A4000419B1
:10281800266A0727B0460F261F40BF00BE40370074
:102828004646BE4326628468AC4384604468944349
:102838004460C268AA43C2600A000133DA4019D072
:102848004A460F009A4017401142F5D0134D9C0894
:10285800A846A4005D464444266E01940F241D40FA
:10286800ED00AC40A0462640A024E405A042A2D139
:102878000025ACE703B0F0BCBB46B246A946A0466B
:10288800F0BD4C46AC402500A1E70224AC40250031
:102898009DE75C46AC40250099E7C0460018024019
:1028A8000004005000080050000C00500069084067
:1028B800431E9841C0B27047002A01D08161704719
:1028C8008162FCE7426913000B401B0491431943E2
:1028D800816170470B4B10B5DA680400104204D1CF
:1028E800084B1A69224207D110BDD86002F06CFB70
:1028F800044B1A692242F7D020001C6102F01CFC2C
:10290800F2E7C0460018024070B5041E23D00368E1
:10291800154A1A60154A1A6042685A6082689A60B5
:10292800FEF7DAFD23680600DA6852070CD007259F
:10293800FEF7D2FD2368801B312802D9DA681542D8
:102948000BD1DA681542F3D11969E268914206D0D1
:1029580000201A6170BD0120FCE70320FAE7044A51
:1029680000201A60F6E7C046CCCC000055550000A0
:10297800AAAA00000368024A00201A607047C046ED
:10298800AAAA000070B5134C134A23680025134007
:102998000343236080239B00984201D0280070BD28
:1029A8000E4B0F491B685800C0184000FDF7A4FBE8
:1029B80080226369D2000130134202D1EEE7002879
:1029C80005D0636901381342F9D10025E6E70325EC
:1029D800E4E7C04600700040FFF9FFFF0000002058
:1029E80040420F00F0B5CE46474680B5040083B09C
:1029F800002800D1F5E00368DA0731D53822C84944
:102A08008868C9680240102A00D1F0E0082A00D17D
:102A1800F1E0802263685202934200D1FEE0A021D7
:102A2800C9028B4200D1D2E1BD4DBE492A680A4095
:102A38002A602A68BC490A402A60002B00D0F1E0CD
:102A4800FEF74AFD80270600BF0205E0FEF744FDB9
:102A5800801B642800D939E12B683B42F6D12368F2
:102A68009A072CD53823AE4A91680B40D168102BB1
:102A780000D1E8E0002B00D0EAE013685B0500D540
:102A8800ABE051686369A9481B0201400B435360DE
:102A9800A34AA74913680B4021690B4313601368C5
:102AA800A44A9B045B0FDA401300A34A1360A34BAC
:102AB8001868FEF7CBFC002800D092E023681A07BC
:102AC8006DD45B0745D53823954A91680B40202B78
:102AD80000D1E3E080230020D16B5B0581461942D9
:102AE80008D1D16B1943D163D26B13400193019B79
:102AF800012399468027924E7F0033683B4200D1DC
:102B0800D5E0A368012B00D124E1052B00D1BBE15E
:102B18000121834EF26D8A43F265F26D03318A43D7
:102B2800F265002B00D019E1FEF7D6FC022307005E
:102B38009846844D05E0FEF7CFFCC01BA84200D99B
:102B4800C4E04246F36D1A42F5D14B46012B00D141
:102B580056E1E369002B20D03822714DA9680A405C
:102B6800102A00D10CE1022B00D14FE12B68764AE4
:102B7800802613402B60FEF7AFFCB604040005E086
:102B8800FEF7AAFC001B022800D99FE02B683342FD
:102B9800F6D1EB686D4A1340EB60002022E0382242
:102BA8005F4DA9680A40182A2FD0A369002B00D1CD
:102BB8008EE001222B6E022713432B66FEF78CFC56
:102BC800060005E0FEF788FC801B022800D97DE09E
:102BD8002B6E1F42F6D0236873E7E368002B00D002
:102BE8004FE7012003B0C0BCB946B046F0BDC943A9
:102BF8008A0700D00DE74A4A1268920300D42FE7EB
:102C08006268002A00D02BE7EBE72A6E920700D40F
:102C180057E7A269002A00D053E7E2E7404A116863
:102C28000B431360FEF758FC802605003C4FB602A4
:102C380004E0FEF751FC401B642847D83B68334248
:102C4800F7D023680CE70D3B0B40022B00D1C8E0FE
:102C5800E368334D002B4ED02B68354A802713404C
:102C68002269FF0013432B6080232A685B0013430B
:102C78002B60FEF731FC060004E0FEF72DFC801BFC
:102C8800022823D82B683B42F7D06A686369274932
:102C98001B020A4013436B60236810E7D36D9B0740
:102CA80000D456E7A368002B00D052E799E73368B1
:102CB8003B433360FEF710FC050033683B4200D00D
:102CC8001FE7FEF709FC401B0228F6D9032089E715
:102CD80001222B6E022793432B66FEF7FDFB0600AD
:102CE80004E0FEF7F9FB801B0228EFD82B6E1F4289
:102CF800F7D12368E5E62B68154A802713402B6037
:102D0800FEF7EAFBFF00060004E0FEF7E5FB801B88
:102D18000228DBD82B683B42F7D12368CFE6C046B0
:102D280000100240FFFFFEFFFFFFFBFFFF80FFFFD9
:102D3800FFC7FFFF0024F400000000200800002067
:102D48000070004088130000FFFFFFFEFCFFFEEF4D
:102D5800FFFEFFFF5149CA6D1343CB65FEF7BCFB6D
:102D68004E4B0600984602274D4D04E0FEF7B4FB93
:102D7800801BA842AAD84346DB6D1F42F6D0E4E682
:102D8800012B00D12DE70323EA68216A13408B4207
:102D980000D026E77023616A13408B4200D020E7F9
:102DA800FE21A36AC90111401B02994200D018E70D
:102DB800F823E16A9B0313408B4200D011E7236B91
:102DC800520F52079A4200D00BE700200AE78021F1
:102DD800324BC90218680143196019680A431A601E
:102DE80020E713685B0503D5E368002B00D1F8E6FC
:102DF800516863692B481B0201400B43536056E638
:102E0800264A2949D36B0B40D363A2E62B68274A8D
:102E1800802713402B60FEF75FFBBF04060005E028
:102E2800FEF75AFB801B022800D94FE72B683B426C
:102E3800F6D1616A236AEA680B431D49174E0A40B6
:102E48001343E26A1343226B1343A26A1202134329
:102E5800EB6080232A685B0413432B608023EA68B5
:102E68005B051343EB60FEF737FB80250400AD04D8
:102E780005E0FEF731FB001B022800D926E733687E
:102E88002B42F6D00020ADE60421044BDA6D0A434C
:102E9800DA65DA6D03390A43DA655FE70010024044
:102EA80088130000FF80FFFFFFFFFFEFFFFFFFFE1B
:102EB8008C80C11F3823204A10B591680B4205D178
:102EC80013681E489B045B0FD84010BD91681940D9
:102ED800082911D09168194010290FD0916819401C
:102EE800202921D090681840183843425841FA23C5
:102EF8004042DB011840E8E71148E6E7D368D168AB
:102F0800DB43D0684906490F40040131440E9B0752
:102F18000DD00A48FDF7F0F86043074BD968490F10
:102F28000131FDF7E9F8D0E780200002CDE7044839
:102F3800FDF7E2F86043F0E7001002400024F400D7
:102F480000127A00F8B5CE46474605000C0080B559
:102F5800002826D00722574E336813408B425ED391
:102F68002B689A070ED55A0705D5E0225249D20197
:102F7800886802438A60504950488A680240A868B5
:102F880002438A60DB072BD56B684B4A012B00D1C3
:102F98007CE0022B07D0002B00D07DE012685205A0
:102FA80004D4012037E012689201FAD50721424E75
:102FB800B2688A431343B360FEF78EFA3823984603
:102FC8003F4B0700994604E0FEF786FAC01B4845C8
:102FD8003BD84346B2681A406B68DB009A42F3D18B
:102FE8000722344E33681340A34238D82B685B0756
:102FF8002DD4FFF75FFF304B324A9B681B051B0F30
:103008009B009B581F221340D8402F4B18602F4B12
:103018001868FEF71BFAC0BCB946B046F8BD33685D
:1030280093430B433360FEF757FA07239846244B24
:1030380007009946424633681340A34200D18FE700
:10304800FEF74AFAC01B4845F4D90320E3E71A4AB9
:103058001F4993680B40E9680B439360C9E73368DD
:10306800934323433360FEF737FA07239846144BFC
:1030780007009946424633681340A342B6D0FEF78C
:103088002BFAC01B4845F5D90320C4E71268920300
:1030980000D58BE70120BEE7032B05D0D26D920740
:1030A80000D583E70120B6E7126E920700D57DE7C9
:1030B8000120B0E70020024000100240FFF0FFFFAF
:1030C8008813000028600008000000200800002085
:1030D800FF8FFFFF064B074A9B685B045B0F9B0053
:1030E8009B581F221340044A1068D8407047C046B6
:1030F800001002406860000800000020F0B5CE46CD
:10310800474680B50368040083B000209A034FD572
:103118008022514B5205D96B8046114200D178E08C
:1031280080274E4D7F002B683B432B60FEF7D4F978
:10313800060005E0FEF7D0F9801B022800D972E0EE
:103148002B683B42F6D0444DC023EA6D9B0011002A
:1031580019401A4220D0606988421ED08022E96D49
:10316800EE6D52023243EA65EA6D3D4B3D4E0B402F
:103178003240EA65EB65CB076CD5FEF7ADF93A4B03
:1031880006000227994604E0FEF7A6F9801B484589
:1031980049D8EB6D1F42F7D061692F4A3048D36D8B
:1031A80003400B43D36543460020012B3FD02368DF
:1031B800DA0706D5032528494A6DAA4365682A43D4
:1031C8004A659A0606D52449284D4A6D2A40A568BD
:1031D8002A434A655A040AD51F4925694A6D92004F
:1031E80092082A434A658022D205954226D01B05BB
:1031F8000AD5194AE168536D1D4C23400B435365AA
:103208008023DB0199421FD003B0C0BCB946B04649
:10321800F0BDD96B1143D963DB6B1A400192019B56
:10322800012398467CE743460320012BBFD10A4A75
:103238001049D36B0B40D3632368B9E78022CD686C
:1032480052022A43CA60D2E78023D1685B020B434B
:10325800D360D9E70100A0E70010024000700040E9
:10326800FFFCFFFFFFFFFEFF88130000FFCFFFFFFB
:10327800FF3FFFFFFFFFFFEF10B5041E5FD03D23A8
:10328800C35CDAB2002B4CD03D230222E254226800
:103298002C4913688A4215D02B498A4246D02B49BB
:1032A8008A4247D02A498A4210D02A498A420DD0F8
:1032B80080218B43A1690B431360E368D362636881
:1032C800936212E070218B43A1680B4322490B40A3
:1032D80021690B4380218B43A1690B431360E36889
:1032E800D36263689362636913630123536148225D
:1032F8000020A3540A3AA3540132A3540132A35420
:103308000132A3540132A3540132A3540132A3540D
:103318000132A3540132A3540132A3540A3AA354EC
:1033280010BD3C33C254FDF75DFFADE770218B4300
:10333800A1680B4308490B4021690B43B8E70120FA
:10334800EEE7C046002C0140000400400020004089
:103358000044014000480140FFFCFFFF3D22815C22
:103368000300012001290FD1013199541B68DA6843
:103378000243DA600D4A934207D00D4A934204D0C3
:103388001A6810431860002070479A6809490A4073
:10339800062A08D007398A4205D001211A68002078
:1033A8000A431A60F0E70020EEE7C046002C01400F
:1033B80000040040070001007047C04610B5041E15
:1033C8005FD03D23C35CDAB2002B4CD03D230222F0
:1033D800E25422682C4913688A4215D02B498A4244
:1033E80046D02B498A4247D02A498A4210D02A49D6
:1033F8008A420DD080218B43A1690B431360E36897
:10340800D3626368936212E070218B43A1680B4317
:1034180022490B4021690B4380218B43A1690B434F
:103428001360E368D362636893626369136301237B
:10343800536148220020A3540A3AA3540132A354EA
:103448000132A3540132A3540132A3540132A354CC
:103458000132A3540132A3540132A3540132A354BC
:103468000A3AA35410BD3C33C254FFF7A5FFADE799
:1034780070218B43A1680B4308490B4021690B431A
:10348800B8E70120EEE7C046002C014000040040E8
:10349800002000400044014000480140FFFCFFFFBD
:1034A80010B500292BD13E23C25C012A25D1022464
:1034B800C4540368DA682243DA601F2211401E3AB6
:1034C8008A40196A91431962196A0A431A62364A8C
:1034D80093422AD0354A934236D0354A934233D064
:1034E800344A934226D0012100201A680A431A6000
:1034F80010BD4023C35C012B44D00120F8E7042908
:1035080035D00829F5D00C2924D0102943D04322DE
:10351800835C012BF1D1082934D00C291ED0102945
:103528003DD0022383540120E2E78022596C120225
:103538000A435A649A6820490A40062A02D0073981
:103548008A42D0D10020D3E78022596C12020A4364
:103558005A64C5E74123C35C012BCED14123022223
:10356800C25403681020DA680243DA60A5E73F23F3
:10357800C25C012AC1D10222C2540368DA680A4334
:10358800DA609AE740230222C25403680820DA6806
:103598000243DA6091E74223C35C012BADD1422399
:1035A8000222C2540120A3E7002C0140004401403C
:1035B80000480140000400400700010003003C20CF
:1035C800F0B51C5C012C00D16CE101241C54142AB8
:1035D80003D8B54892008258974601203C22002122
:1035E8009954F0BD1A68B14C106AB14D2040106270
:1035F800106A5668546D2C400D682D022543AD4C59
:103608000440886800052043AB4CA24200D111E178
:10361800AA4CA24200D10DE1A94CA24200D109E175
:103628004C6856605565D46510628020546D000161
:1036380020435065506DA34C096920405065506D7A
:103648000902014351650020C8E701241A689E4F0A
:10365800106A0D68A0431062106A566894693C406D
:1036680002272C43B8438D68934F2843BA4200D1B0
:103678000BE1924DAA4200D107E1914DAA4200D137
:1036880003E1566094614C68096954630824106228
:103698009069204390619069043CA04390619069CF
:1036A80001439161002099E710241A68874D106A38
:1036B800814FA0431062106A566894692C400D68C7
:1036C8002D0225432024A0438C6824010443BA42D8
:1036D80000D1CAE0794FBA4200D1CEE0784FBA4261
:1036E80000D1CAE0486856609561906380201462F2
:1036F80094690001204390619069724C09692040E7
:1037080090619069090201439161002066E71A6897
:103718006F4C106A6C4E20401062106A5568D4696C
:103728000F68344027436B4C634E20408C6824025A
:103738000443B24200D189E0604EB24200D18CE02D
:103748005F48824200D188E048685560D761D063FD
:1037580014620824D06909692043D061D069043C07
:10376800A043D061D0690143D161002036E71A68CF
:10377800594C106A554D20401062106A5668D46939
:103788002C400D682D022543544C044088680003E2
:103798002043494CA24253D0484CA24250D0484CF6
:1037A800A2424DD04C685660D561146410628020E6
:1037B800D46900012043D061D069424C0969204096
:1037C800D061D06909020143D161002006E71A6877
:1037D800434C106A434D20401062106A5668546D7D
:1037E80025400C682543404C044088680004204369
:1037F800314CA24218D0314CA24215D0304CA242D2
:1038080012D04C6856605565946508241062506D56
:10381800096920435065506D043CA0435065506DC4
:10382800014351650020D9E62D4C34404E693602DB
:103838002643E6E72D4C34404E69B6022643EFE6B0
:103848002B4C34404E69B6012643ABE7294820404B
:10385800CC68240204431B48044027484E6928408A
:103868008D6935432D0105436EE780208443200090
:10387800CC68240104434020844320484F693040E9
:103888008E693E43B60006432CE70825A843CD6859
:103898008F6928430425A843194D35404E693E4396
:1038A8002E43EEE602209CE688600008FFFFEFFF4B
:1038B800FF8FFFFEFFFFDFFF002C014000440140A7
:1038C80000480140FFFBFFFF8CFFFEFFFF8CFFFE5F
:1038D800FFFEFFFFFFFDFFFFFFEFFFFFFFDFFFFF23
:1038E800FFFFFEFF8FFFFEFFFFFFFDFFFFFFFBFF58
:1038F800FFBFFFFFFFF7FFFFFFCFFFFFFFF3FFFF54
:10390800FFFCFFFF70B5041E18D088262423012170
:103918000025835103681A688A431A601D605D6038
:103928009D60FDF745FD90230020E550043BA5511F
:10393800E550083BE5662567E55470BD0120FCE7C6
:10394800F8B51300882282580400202A41D10029A2
:103958002CD0002B2AD0802280685201904220D09F
:1039680054222165A3520232A3522120902600221C
:103978008825A2516051E06F002819D0164F826344
:10398800C762164F22680763154F28324763FEF750
:103998002BFB00280CD01023A351103301206351B6
:1039A80005E02269002ADBD1CA07D9D50120F8BD74
:1039B800402223681A62EFF31081012383F31088F1
:1039C8008020226893680343936081F31088002065
:1039D800EDE70220EBE7C046293C00087D3C0008E3
:1039E800953C0008F8B504008C202058202800D009
:1039F8006DE0002942D0002A40D08023A0685B01F6
:103A0800984205D12369002B02D10120CB0736D477
:103A18000023E36623685B681B020CD5EFF310856F
:103A2800012383F3108880232068DB04066833436E
:103A3800036085F310885C23A1652220E25290265A
:103A480000238C25A35160515E302058002817D0E0
:103A5800204F8363C762204F130007631F4F0A007C
:103A68004763276824373900FEF7BEFA002807D0D5
:103A78001023A35110330120635100E00120F8BD49
:103A88002369002B0BD0EFF31081012383F31088F7
:103A98002268FF3310680343136081F31088EFF343
:103AA8001080012383F3108821688A681A438A608A
:103AB80080F31088EFF3108183F310884020226888
:103AC80093680343936081F310880020D7E70220AE
:103AD800D5E7C0467D4100085D410008953C0008D7
:103AE800882370B504008022C0580433E558236841
:103AF80099680A4201D0212807D09A6840230020FB
:103B0800134201D0222D33D070BDEFF31080012372
:103B180083F3108821688B6893438B6080F3108847
:103B2800E06F002803D0FEF7C7FA00286AD1EFF348
:103B38001080012282F31088C02621680B68B343E5
:103B48000B6080F31088EFF3108182F310882268ED
:103B58002F4893680340936081F3108888232022BC
:103B6800E250236800209A6840231342CCD0C9E76A
:103B7800EFF31080012282F3108821688A689A4343
:103B88008A6080F310885E356059002803D0FEF7FC
:103B980093FA00282CD1EFF31080012282F31088C9
:103BA80021681C4D0B682B400B6080F31088EFF3E5
:103BB800108182F310882268174893680340936045
:103BC80081F31088E36E012B0AD1EFF3108183F3A0
:103BD80010881020226813688343136081F31088CB
:103BE8008C232022E25000230020E36663678BE7E2
:103BF8006059FEF73DFB2028CDD1902310221D38B7
:103C0800E25081E7E06FFEF733FB20288FD1F4E71D
:103C1800FFFF7FFFDFFEFFFFFEFFFFEF7047C0469D
:103C28002022030011001B6810B51B68806A194028
:103C38001A4219D15623C152EFF3108C1F3A82F35E
:103C48001088802401688B68A3438B608CF31088EC
:103C5800EFF3108182F31088026840201368034351
:103C6800136081F3108810BDFFF7D8FFFBE7C0464B
:103C78007047C04610B5806AFFF7FAFF10BDC0460E
:103C88007047C0467047C0467047C046F8B588229E
:103C98008C23806A8558C45803689968090601D539
:103CA800212D0CD09B685B0601D5222C25D09022B3
:103CB800102183580B438350FFF7E6FFF8BD5623C6
:103CC8000021C152EFF31086013181F31088C0271B
:103CD80005682B68BB432B6086F31088EFF31085CB
:103CE80081F3108801681C4E8B6833408B6085F324
:103CF8001088202383500368D4E75E230022C25231
:103D0800EFF31084013282F310880168134D0B68B9
:103D18002B400B6084F31088EFF3108182F3108836
:103D280002680F4C93682340936081F31088C36E38
:103D3800012B0AD1EFF3108183F310881024026855
:103D48001368A343136081F310888C232022C25088
:103D58000023C3664367AAE7FFFF7FFFDFFEFFFF7D
:103D6800FEFFFFEF00235E2210B5806A8352083AF7
:103D78008352FFF789FF10BD7047C046F8B5454626
:103D8800DE4657464E460268E0B5D369A84D0400A2
:103D9800106891682B4200D1F7E0A64EA64D0E4060
:103DA8000540354357D1E56E012D26D080256D039A
:103DB8002B4202D04E0200D510E180221A4206D0D2
:103DC80080252D0402402940114300D0FFE0402205
:103DD8001A4202D0024200D009E11A0202D542007A
:103DE80000D518E1DB0102D5002800DA6FE1F0BC4C
:103DF800BB46B246A946A046F8BD10261E42D5D0FD
:103E08000642D3D04023180016629268104013422D
:103E180000D119E180229346A2581068426892B2F4
:103E2800002AE4D05C218A46615A9142DFD95E2794
:103E3800E2532022170000680740B846024200D12A
:103E48004EE1022323675C33E35A2000C91A89B282
:103E5800FFF792FFCBE701251D4208D0C70506D51D
:103E68009027BC461562E7593D436746E551022550
:103E78001D4200D198E0CF070CD515628E35042776
:103E8800AC466559B8463D436746E55145461D422F
:103E980000D08FE008271F4208D0202505402E4378
:103EA80004D090261762A5592F43A75180252D01CC
:103EB8002B4207D0460105D5902620271562A55923
:103EC8003D43A55190256559002D00D18FE7202548
:103ED8001D4206D005408020400501400D4300D01A
:103EE8009DE090264025A15993681D4028230B404A
:103EF8001D4300D1EFE0EFF31080012282F3108818
:103F080021684E4D0B682B400B6080F31088EFF34F
:103F1800108182F3108822684948936803409360AF
:103F280081F31088E36E012B0AD1EFF3108183F33C
:103F380010881020226813688343136081F3108867
:103F48008C232022E2500023E36663672368203233
:103F58009B681A4247D0EFF31080012383F310883F
:103F680021688B6893438B6080F3108880256059A3
:103F7800002838D0334B8363FEF7DCF8002800D1E3
:103F880035E76059836B984731E720251D4200D1FA
:103F980009E78026760505400E40354300D102E743
:103FA800636F002B17D122E75D0700D472E7CD07B6
:103FB80000D46FE7042515628C35A9466559A846D3
:103FC800022547462F433D004F46E55162E7A36F60
:103FD800002B00D10BE72000984708E72000156266
:103FE80000F00EFB03E72000FFF74EFEFFE6EFF3BD
:103FF8001080012383F3108821680B6893430B60BA
:1040080080F310888823203AE25000232000A36719
:10401800FFF704FEEBE6200000F0F6FAE7E6636F30
:10402800002B00D15DE720009847226859E7C04679
:104038000F0800000100001020010004DFFEFFFF50
:10404800FEFFFFEF6D3D00085E22A35AA25A9BB205
:10405800002A00D1CBE65C22A15AC91A89B20029EC
:1040680000D1C4E6EFF3108785F3108823689946DA
:104078001B6898464246344B1A4013004A46136060
:1040880087F31088EFF3108785F310882368994623
:104098009B68984642462D4B1A4013004A46936047
:1040A80087F310888C232022E250E0666067EFF3E4
:1040B800108085F3108822681368B343136080F377
:1040C8001088022320002367FFF756FE8FE62000A2
:1040D80000F098FA8BE62000FFF7D6FDA55186E69A
:1040E800EFF3108985F310882068194F016839406B
:1040F800016089F31088EFF3108985F31088206830
:104108008168A943816089F31088EFF3108985F3EA
:104118001088206881689943816089F310884C333E
:10412800E2504346E366EFF3108185F31088226876
:104138001368B343136081F310885B46E058FDF7BA
:10414800BBFF5346E15A7CE6DFFEFFFFFEFFFFEFB1
:10415800FFFEFFFF0123806A10B50367C36E012BC2
:1041680002D0FFF78FFD10BD5B33C15A4908FFF736
:1041780003FEF8E703001B6870B51A6820231900CE
:10418800806A1140134227D15E228152EFF31085D5
:104198005D3A82F3108804681C4E21683140216022
:1041A80085F31088EFF3108582F310880468A168FE
:1041B8009143A16085F31088EFF3108482F310888F
:1041C800402501688A68AA438A6084F310888C2293
:1041D8008350C36E012B0CD000230367C36E012BE1
:1041E80002D0FFF74DFD70BD5B33C15AFFF7C4FD28
:1041F800F9E7EFF3108183F310881024026813683D
:10420800A343136081F31088E6E7C046FFFEFFFF73
:10421800836A30B5DA0706D50168284C4A68224017
:10422800C46A22434A609A0706D50168244C4A6842
:104238002240046B22434A605A0706D50168214C84
:104248004A682240446B22434A601A0706D501682F
:104258001D4C4A682240846B22434A60DA0606D520
:1042680001681A4C8A682240C46B22438A609A0605
:1042780006D50168164C8A682240046C22438A607D
:104288005A060AD50168134D4A68446C2A402243ED
:104298004A6080225203944209D01B0606D5026860
:1042A8000D4953680B40C16C0B43536030BD4A68DD
:1042B8000A4C2240846C22434A60EEE7FFFFFDFF70
:1042C800FFFFFEFFFFFFFBFFFF7FFFFFFFEFFFFF8B
:1042D800FFDFFFFFFFFFEFFFFFFFF7FFFFFF9FFF7E
:1042E800F0B54646984604234F4699468023D6465D
:1042F8001B01C0B5150007009A460C00089E01680E
:10430800731C0CD1CB6923401B1B5A425341AB424F
:10431800F8D00020E0BCBA46B146A846F0BDCB694B
:1043280023401B1B5A425341AB42F2D1FDF7D4F84C
:104338004346C01AB0422DD8002E2BD04A463968C1
:104348000B681A42DCD05246CB691342D8D00A62B5
:10435800EFF31080012282F3108839681A4C0B6839
:1043680023400B6080F31088EFF3108082F31088ED
:1043780039688B6893438B6080F3108820238732D9
:10438800BB500432BB500432BB50002264330320BC
:10439800FA54BFE7EFF31080012282F310883968DE
:1043A800094C0B6823400B6080F31088EFF31080F2
:1043B80082F3108839688B6893438B6080F3108888
:1043C80020238732DEE7C0465FFEFFFF30B50400DA
:1043D80083B0002800D1E1E08823C358002B00D126
:1043E80088E0882324220121E250236825691A687D
:1043F800E0698A431A60A26819682A4365692A43F2
:10440800714D024329400A431A605A686F49256A68
:104418000A40E1680A435A60A26999682A436C4DC8
:1044280029400F250A439A60DA6A616AAA430A4357
:10443800DA62684A93420AD0674A93420ED0674BC1
:104448000120A36600236367A36703B030BD644BF4
:104458005A6D03231340013B022B50D980231B02C2
:1044680098425CD0FEF736FE002812D0616A5D4B98
:104478004900C95AFBF740FE65686B08C018290057
:10448800FBF73AFE0200584B103A9A42D7D82368F5
:10449800D860524BA36600236367A367A36A002B07
:1044A80002D02000FFF7B4FE236850495A680A403A
:1044B8002A215A609A688A439A601A6829390A43F5
:1044C8001A6090230022E250FDF706F823680500E1
:1044D8001A68120746D41B685B0752D42023882227
:1044E800A3500432A3500023083AE3660020236750
:1044F800A354AAE784228354FCF7D2FE71E73C4A0E
:10450800D25C80231B0298424DD0042A48D025D87B
:10451800002AA7D0022A00D091E73648A7E7FEF77D
:10452800D9FD0028B5D0616A2E4B4900C95AFBF75E
:10453800E3FD656840006B08C0182900FBF7DCFD47
:104548000200294B103A9A4200D978E72A4B226890
:1045580003400007400F1843D0609AE71800082A64
:1045680085D06CE78021254B002200938903030046
:104578002000FFF7B5FE00280ED123681B685B07F3
:10458800ACD580211D4B0022009320002B00C903CD
:10459800FFF7A6FE0028A1D0032056E7012054E724
:1045A800FEF788FC60E7042A07D009D8002AB6D0AD
:1045B800022A00D043E70F48B6E7FEF77BFCB0E7D6
:1045C800082AB1D03BE7C046F369FFCFFFCFFFFF12
:1045D800FFF4FF11003801400044004001000100D1
:1045E80000100240E0600008EFFF0000FFB7FFFF87
:1045F800DC6000080024F400F0FF0000FFFFFF016A
:104608007047C0467047C0467047C04670B584249E
:10461800035D012B12D0882524230126435103680A
:104628001A681968B143196005490A4000214166B2
:104638001A60202343510155002070BD0220FCE779
:10464800FFFFFFDFF0B5D6464F4646468423C0B588
:10465800C35C04000A00012B3DD08823242105688F
:10466800C1502E682B6823398B432B60AB68DB0065
:10467800D908436E1143A960002B29D0AB68174AAB
:1046880098469246AB685B0FD05C154AC000D15C77
:104698009146FBF7BBFD434652461B015B0F87B2B1
:1046A800D05C4A46C000D15CFBF7B0FD80B26823FD
:1046B8002022E0520233E7521E332E60E2500022DD
:1046C8000020043BE254E0BCBA46B146A846F0BD1F
:1046D80001200127EBE70220F5E7C046006100084A
:1046E800F8600008F0B5D6464F4646468423C0B564
:1046F800C35C04000A00012B3DD0882324210568EF
:10470800C1502E682B6823398B432B60A9681B4B3B
:104718001940436E1143A960002B29D0AB68184A91
:1047280098469246AB685B0FD05C164AC000D15CD5
:104738009146FBF76BFD434652461B015B0F87B260
:10474800D05C4A46C000D15CFBF760FD80B26823AC
:104758002022E0520233E7521E332E60E25000223C
:104768000020043BE254E0BCBA46B146A846F0BD7E
:1047780001200127EBE70220F5E7C046FFFFFFF124
:1047880000610008F860000800230270FA224371F3
:1047980052000B1C914200D2131CC3807047C046C4
:1047A800F0B5C64600B5438804000A339BB243807F
:1047B8000A2B06D94579002D0CD0962B01D9012D4D
:1047C8002ED0E2889A4202D200236371638080BCB3
:1047D800B846F0BD0123067843713233038100F0F7
:1047E800ABFF7000C0B201F03BF800F0E9FF012810
:1047F80000D194E0AC2001F033F800F0E1FF01288B
:1048080000D196E0207A01F02BF800F0D9FF607A09
:1048180001F026F800F0D4FF00F0B0FF2571D6E7CC
:10482800022306784371050000F086FF700001300E
:10483800C0B201F015F800F0C3FF1C3506000128CE
:1048480000D1A5E02323270098462E00A044223754
:10485800B81BC0B201F038F830700136B045F7D156
:1048680000F08CFF00232000237131212230FF3318
:1048780027E05AB2DEB2002A2EDB7200D3B252B25F
:10488800002A2FDB5A00D3B252B2002A30DB5A007A
:10489800D3B252B2002A31DB5A00D3B252B2002A44
:1048A80032DB5A00D3B252B2002A33DB5A00D3B2F9
:1048B80052B25B00002A00DA4B400135DBB2A84255
:1048C80039D02A7853405AB25B00002AD1DA4B40DB
:1048D8005AB2DEB2002AD0DA73004B405AB2DBB2C9
:1048E800002ACFDA5B004B405AB2DBB2002ACEDA9C
:1048F8005B004B405AB2DBB2002ACDDA5B004B407A
:104908005AB2DBB2002ACCDA5B004B405AB2DBB2B7
:10491800002ACBDA5B004B405AB2DBB2C9E7AC20C5
:1049280000F09EFF00F04CFF012801D0012573E73D
:104938000220050070E72222A25C9A4200D046E7D6
:104948006722237F9343182B00D040E7637FA07F23
:104958001B02C018E57F000228180009FCF74EF872
:104968000F49FBF757FD20630F2020222840030240
:10497800A05CC0182123E35C00021818FCF73EF87D
:104988000849FBF747FD0849FBF76AFE60631EE725
:1049980000F0F4FE002326712363636317E7C04623
:1049A8000000C83800004839000048421021074B71
:1049B80010B51B6806481A680A431A605022EA3183
:1049C8001A62C900183AFFF7DFFE10BD0C0200207A
:1049D800C0020020F0B5C6463C4D00B52888AB1C87
:1049E8000100F535FF351A888A424FD8141C8242D7
:1049F80000D9041CA0B202339D42F4D10B1A002B3B
:104A080004DD334B1A888918091A1980314C237828
:104A18005A1C2270032B36D92F4B2D4E1D882F4B35
:104A280005211B882DB21BB298462D4B1F780023F9
:104A3800F05EFBF7EBFB03B22A482B495843FBF720
:104A4800E5FB0A216843FBF7E1FB03007FB243441F
:104A58007B43264A1BB21380254B1978012926D09F
:104A68001B78002B28D0234A002333802370138817
:104A78001BB2D9175B184B401F499BB28B4207D911
:104A880096221E4B1A8080BCB846F0BD1100B2E7D2
:104A980013881BB2DA179B185340FA229BB25200B4
:104AA80093420ED9154B913AFF3A1A80EBE71388D7
:104AB800104A1BB21380D7E71388114A1BB2138020
:104AC800D1E728220D4B1A80DDE7C046FC02002002
:104AD800F00500200B060020F4050020F205002058
:104AE80017000020E40C0000FF0F0000F60500206E
:104AF800FF050020FA050020DC0500001400002056
:104B0800F8050020F0B557464E464546DE46E0B566
:104B1800B84F8BB0BE887D8876BAB3B26DBA0193B0
:104B28003A000123B44CB549ADB2B81D18E0640889
:104B380023421ED16408234220D16408234222D193
:104B48006408234224D16408234226D164082342FE
:104B580028D1640823422AD10132640890422CD01B
:104B6800167874402342E2D064084C40A4B2234231
:104B7800E0D064084C40A4B22342DED064084C4024
:104B8800A4B22342DCD064084C40A4B22342DAD059
:104B980064084C40A4B22342D8D064084C40A4B264
:104BA8002342D6D064084C40A4B22342D4D064082F
:104BB8004C400132A4B29042D2D1230A9946904B7C
:104BC800E4B21A888F4B5A808F4A127852B29A8070
:104BD8008E4A1278DA808E4A12881A818D4A128893
:104BE8005A818D4A12889A818C4A1288DA818C4AB5
:104BF80012881A828B4A11788B4A090212780A4362
:104C08005A82019A52190A2A02DCBA79A24241D080
:104C1800FF2D06D00BB0F0BCBB46B246A946A04655
:104C2800F0BD019B012BF5D1BB79A342F2D1FB79F1
:104C38004B45EFD105AA11007C4B31CB31C1186827
:104C480008609B888B807A490023080003E0D15CC8
:104C5800C1540133DBB2112BF9D18046A0200122C7
:104C68002021C005FDF728FE112241467148FEF7B4
:104C780067FE714B1C002000FDF7F6FA0128FAD1F7
:104C8800043001F033F9A02000222021C005FDF7EF
:104C980013FEBFE7FA794A45BAD1654A90464146BC
:104CA80040463A880A8001994A008270002900D15A
:104CB80099E041460020A0460322AB460C00594625
:104CC80041184900595E8A4656465546511CC9B294
:104CD8003612A6546554411C019D1600C8B2023212
:104CE800D2B2A842EBD3230044469846330003339C
:104CF800DBB2039333005D46501E043380B2029248
:104D0800DEB23D4BA446AA4601219B4644461D00FF
:104D18003A4A1DE05B08194223D15B08194225D1A4
:104D28005B08194227D15B08194229D15B0819424F
:104D38002BD15B0819422DD15B085D08194202D0BE
:104D48005B0853409DB2013880B20134584525D0E4
:104D580023786B401942DDD05B0853409BB219425F
:104D6800DBD05B0853409BB21942D9D05B08534053
:104D78009BB21942D7D05B0853409BB21942D5D099
:104D88005B0853409BB21942D3D05B0853409BB297
:104D98001942D1D05B0853409BB2CEE72B00424664
:104DA800A0200299C005535403991B0A53540122A9
:104DB80020216446FDF780FD320041461D48FEF77C
:104DC800BFFD1D4B55461E003000FDF74DFA01286A
:104DD800FAD1043001F08AF8A02000222021C00571
:104DE800FDF76AFD14E704230393013B052602201F
:104DF800029386E714060020FFFF000001A0FFFFD2
:104E0800F6050020980600200C000020160000205F
:104E18000E060020F4050020F205002008060020F8
:104E2800FC0500200006002010060020086100088C
:104E3800700500200C020020B0010020002310B5EE
:104E48008AB000210C2207A8069301F0B4F80222C8
:104E58000423029203930F22012304920593234B08
:104E680006AC1A881B8822701B0A6370204B1A88AC
:104E78001B88A2701B0AE3701E4B1A881B882271BC
:104E88001BB21B1263711C4B1A881B88A2711BB2C0
:104E98001B12E371194B1A881B8822721BB21B1252
:104EA8006372FDF7AFFA01A902A8FDF7FFFA00281F
:104EB80018D1069A079B01201149FDF7DBF9002854
:104EC8000CD1089A099B01200E49FDF7D3F9041E5D
:104ED80004D1FDF7A9FA20000AB010BDFDF7A4FA25
:104EE8000324F8E7FDF7A0FA0124F4E7FA0200200A
:104EF8000E060020F4050020F2050020FC05002025
:104F080000780008087800080222042310B586B04B
:104F1800029203930E220123154C049205932368F1
:104F280008332360FDF76EFA2168124B994208D9BD
:104F3800114B01A902A82360FDF7B8FA00280ED189
:104F480021680E4B01201A88002392B2FDF792F9CE
:104F5800041E08D1FDF768FA200006B010BDFDF761
:104F680063FA0124F8E7FDF75FFA0324F4E7C04683
:104F780010000020D87700080070000808060020FC
:104F880010B50400A02001222021C005FDF794FCE3
:104F9800A2B20A490A48FEF7D3FC0A4C2000FDF7E2
:104FA80063F90128FAD1043000F0A0FFA020002204
:104FB8002021C005FDF780FC10BDC046700500200B
:104FC8000C020020B0010020F0B5C6460400A02065
:104FD800402100B5C005FDF769FC484D80212870C7
:104FE800A020C005FDF762FC802C06D0082C24D038
:104FF800434BDC6080BCB846F0BD0128F8D1FCF713
:105008006BFA404F06003B68C31A072B5FD92B7811
:105018003E60012B56D03C4A13780133DBB2137043
:10502800092BE5D9394B1978022963D90120384968
:105038000870002111701970DAE70320354900F073
:1050480019FFA0200821C005FDF730FC0128CFD1A9
:10505800314B3249324A1870324D0B8812882D88EC
:105068001BB212B29B1AAB421DDC2F4A13780133D4
:10507800DBB21370012B08D92C4D287000252C4861
:105088000570FA2B01D9032313700B881BB2DA17AA
:105098009B185340FA229BB252009342A8D8002290
:1050A800224B1A70A4E7224A13780133DBB213703B
:1050B800012BEAD900201D4D28701B4D2870FA2BB2
:1050C800E1D8E2E7114A137801331370A3E7FA2114
:1050D8000420890000F0CEFE164B98461B78012B61
:1050E80095D1FA210220490000F0C4FE002342466F
:1050F80013708CE7FF20064908709AE7F802002031
:105108000018024004060020FE0500200C060020BE
:105118001700002088130000FF050020FA05002072
:10512800F8050020140000200A0600200C000020CA
:105138000D0600201600002010B5082800D010BD6C
:10514800A0200821C005FDF7B1FB0028F7D1014BCD
:105158001870F4E7FF05002070B5284C0500200002
:10516800FEF7D0FB264B2360012D37D0022D31D01E
:1051780096239B01636000230C222000A360E36058
:1051880023616261A361E36123626362A362FFF743
:105198001DF900282FD100212000FFF753FA00281D
:1051A80026D100212000FFF79DFA00281DD12000FC
:1051B800FFF72CFA002815D11021236811481A6826
:1051C8000A431A60FA215022C9001A62183AFFF7F6
:1051D800DBFA70BDE1231B026360CCE79623DB0199
:1051E8006360C8E7FBF720FFE6E7FBF71DFFDEE794
:1051F800FBF71AFFD5E7FBF717FFCCE70C020020F7
:1052080000380140C0020020F0B54E464546DE4653
:105218005746E0B5A34C0122A588A0466BBA9B4629
:105228009BB29946638821005BBA9F4D9F4887B01F
:105238009EB2A71D1BE05B081A4221D15B081A42E7
:1052480023D15B081A4225D15B081A4227D15B0893
:105258001A4229D15B081A422BD15B085D081A4211
:1052680002D05B0843409DB201318F4225D00B78B4
:105278006B401A42DFD05B0843409BB21A42DDD034
:105288005B0843409BB21A42DBD05B0843409BB2A9
:105298001A42D9D05B0843409BB21A42D7D05B0868
:1052A80043409BB21A42D5D05B0843409BB21A4296
:1052B800D3D05B0843409BB2D0E77D4B22689A4627
:1052C8001A6051465246A3889380EBB22A0ACD80D1
:1052D8000F2E00D1D1E0042E55D0594608B2052E24
:1052E8005CD0062E00D18DE0072E00D0A8E0A17971
:1052F80099424CD1E379934249D15B466D4C0222E5
:10530800268823800423029203930E2201236A4DE8
:1053180004920593694BB6B22B60FDF773F82968C0
:10532800674B994209D9674B01A902A82B60FDF781
:10533800BDF8002800D0A6E12968228800230120B2
:1053480092B2FCF797FF002800D09CE1FDF76CF8BB
:10535800A02001222021C005FDF7AEFA08225146FF
:105368005948FEF7EDFA594C2000FCF77DFF01285B
:10537800FAD1052000F0BAFDA02000222021C005A6
:10538800FDF79AFA03E0A179994200D1F3E007B05A
:10539800F0BCBB46B246A946A046F0BDA1799942E9
:1053A800F5D1E3799342F2D1494B4A4A4B449BB237
:1053B8009342ECD8484C494B278819888300181821
:1053C80009B24000FAF722FF4E4600B2053E3FB24E
:1053D80020800F2E01D85B46238023881BB2042B24
:1053E800D5DD23881BB2142BD1DC012383F310886D
:1053F800FFF724FD002383F31088002800D14AE139
:105408002780C4E7A1799942C1D1E3799342BED1FB
:105418002F4E304B4E44B6B29E42B8D85B46304C05
:105428002688238036B2012383F31088FFF706FD10
:10543800002383F31088002800D1D5E02680A6E752
:10544800082EA4D1A1799942A1D1E37993429ED1A2
:105458004B46032B9BD85B46224E3488338024B2BC
:10546800012383F31088FFF7E9FC002383F31088F6
:10547800002800D113E1348089E7A179994200D04E
:1054880085E7E379934200D081E74E46013EF62E48
:1054980000D8D3E0012352465B429380034901229E
:1054A800014B3CE014060020FFFF000001A0FFFFB5
:1054B800700500200806002010000020E077000892
:1054C800D8770008007000080C020020B001002006
:1054D800E40C0000C8190000F4050020F6050020BF
:1054E800F2050020FC0500205B081A4221D15B0868
:1054F8001A4223D15B081A4225D15B081A4227D1E8
:105508005B081A4229D15B081A422BD15B081A4260
:105518002DD15B0801208446E044474576D04046BB
:10552800007843401A42DFD05B084B409BB21A42D6
:10553800DDD05B084B409BB21A42DBD05B084B4086
:105548009BB21A42D9D05B084B409BB21A42D7D0C3
:105558005B084B409BB21A42D5D05B084B409BB2CC
:105568001A42D3D05B084B409BB21A42D1D05B0899
:105578004B409BB2CEE7E379934200D007E7FA238A
:105588009B00994500D902E75B46544E3488338026
:10559800A4B2012383F31088FFF750FC002383F3A0
:1055A8001088002800D066E7A02001222021C0052D
:1055B800FDF782F9082251464948FEF7C1F9494CDE
:1055C8002000FCF751FE0128FAD1043000F08EFCCF
:1055D800A02000222021C005FDF76EF9424A338839
:1055E80012689BB25363D2E6A02001222021C00595
:1055F800FDF762F9082251463948FEF7A1F9394CFE
:105608002000FCF731FE0128FAD1B2E65246D380D9
:105618002378002B00D1BAE6A02001222021C00562
:10562800FDF74AF9082251462D48FEF789F92D4C15
:105638002000FCF719FE0128FAD19AE65B462B4EAA
:1056480037883380BFB2012383F31088FFF7F6FB56
:10565800002383F31088002819D16378002B00D128
:1056680095E6A02001222021C005FDF725F9082292
:1056780051461B48FEF764F91A4C2000FCF7F4FD6C
:105688000128FAD175E6FCF7CFFE26807FE6FF23D6
:105698003B4033807BE60830FFF772FC77E6A020BA
:1056A80001222021C005FDF707F9082251460C48C0
:1056B800FEF746F90B4C2000FCF7D6FD0128FAD17D
:1056C800043000F013FCA02000222021C005FDF7C3
:1056D800F3F8308800B2FFF73FFD58E60E060020C9
:1056E8000C020020B001002008010020FA0200206E
:1056F80010B50E4B0E4A18781288904206D0002832
:1057080003D10C4A1278082A0AD010BD094A127827
:10571800082AF4D15B78032B03D1FFF7F3F9F4E7F8
:105728005B78062BF1D1FFF76FFDEEE7140600203A
:10573800FA0200209406002070B58026A024802557
:10574800E405760131002D0120000122FDF7B4F8AF
:10575800290001222000FDF7AFF8042000F0DEFB4D
:10576800310000222000FDF7A7F8042000F0D6FB46
:10577800290000222000FDF79FF870BD70B5802633
:10578800A0248025E405360131006D0120000022A7
:10579800FDF792F8290000222000FDF78DF804207B
:1057A80000F0BCFB310020000122FDF785F829003C
:1057B80001222000FDF780F8042000F0AFFB70BD47
:1057C8008021A02070B501224901C005FDF774F8B9
:1057D800012000F0A3FB8021A02001220901C005BF
:1057E800FDF76AF8012000F099FB652403E0013C0D
:1057F800E4B2002C10D08021A0204901C005FDF79B
:1058080055F8051EF3D18021A02000220901C0050A
:10581800FDF752F8280070BD8021A0200022090160
:10582800C005FDF749F88021A02000224901C005E4
:10583800FDF742F8042000F071FB8021A02001222E
:105848000901C005FDF738F88021A020012249018F
:10585800C005FDF731F8042000F060FB0125D9E709
:1058680070B580210400A02000220901C005FDF7C1
:1058780023F8082563B20122002B00DB00228021D7
:10588800A0204901C005FDF717F8022000F046FBEB
:105898008021A02001220901C005FDF70DF8022092
:1058A80000F03CFB8021A02000220901C005013D39
:1058B800FDF702F864000220EDB200F02FFBE4B21D
:1058C800002DD7D170BDC04670B50600082500244C
:1058D8008021A02000220901C005FCF7EDFF02206D
:1058E80000F01CFB8021A0200901C0050122FCF763
:1058F800E3FF8021A02064004901C005E4B2FCF761
:10590800D5FF002801D00134E4B2013D0120EDB2F9
:1059180000F004FB002DDBD18021A020002209012A
:10592800C005002E25D1FCF7C7FF8021A020012249
:105938004901C005FCF7C0FF042000F0EFFA802100
:10594800A0200122C0050901FCF7B6FF042000F0E1
:10595800E5FA8021A02000220901C005FCF7ACFF70
:105968008021A02001224901C005FCF7A5FF2000E5
:1059780070BDFCF7A1FF8021A02000224901C005CD
:10598800FCF79AFF022000F0C9FA8021A02001222A
:10599800C0050901FCF790FF0220D8E7F8B5DE46FC
:1059A80057464E464546E0B5FFF700F8A44B1A881F
:1059B800A44B1A801A88002A00D10EE11988A24A3D
:1059C800914200D109E1A14B1A88A14B1A801A888B
:1059D800002A00D1FDE019889B4A914200D1F8E0E5
:1059E8009C4C1B8822689BB253639B4B00229A5E97
:1059F8009A4B1A801A88002A00D1E7E01A8812B256
:105A0800013200D1E2E0964B00229A5E954B1A8053
:105A18001A88002A00D1D6E01A8812B2013200D1C1
:105A2800D1E0914B00229A5E904B1A801A88002A86
:105A380000D1C5E01A8812B2013200D1C0E018883E
:105A48008B4D00B2FFF788FB002294467E4A894BB3
:105A58009046894E894F18001A880830328032885B
:105A68001989002A00D1E1E03288424500D1DDE001
:105A78004A1E92B2AA4200D8D0E0814A1360338805
:105A88002000FDF76BFC00212000FDF709FD7D4C8F
:105A98002000FEF725F8802220007B49FDF7A2FFB1
:105AA8007A4BFA229A467A4B514618009846FCF7E8
:105AB8006FF8A02000222021C005FCF7FDFE32214E
:105AC800002000F0D7F9FA210120490000F0D2F9AE
:105AD8000320704900F0CEF9FA210420890000F073
:105AE800C9F90A21052000F0C5F96B4B00249B4633
:105AF8006A4B6B4F99466B4D002000F0E5F9002882
:105B080027D1012000F0E0F9002831D1022000F06F
:105B1800DBF900283BD1032000F0D6F9002802D099
:105B280002234A461370042000F0CEF9002868D1F9
:105B3800052000F0C9F9002852D12B78002BDBD0C2
:105B4800FFF7D6FD002300202B7000F0BDF90028D8
:105B5800D7D04046FCF7BAF8FEF73CFFFA22514688
:105B68004046FCF715F8012000F0AEF90028CDD02A
:105B780000234D4A58461380FCF7FCFE4B48012190
:105B8800FCF7A0FE022000F09FF90028C3D0A02057
:105B98000421C005FCF796FEE1230134A4B25B01A1
:105BA8009C42B8D9338801339BB233803288264B64
:105BB8009A4201D100233380FFF7A6F90024AAE70F
:105BC80000221A803BE700221A802AE70A221A805C
:105BD80019E7FA2292001A8002E701221A80F2E6F7
:105BE8003800FEF7DDFD7B79022BA6D1386BFAF77A
:105BF800F9FB2F4B1870786BFAF7F4FB2D4B1870E4
:105C08009BE7022000F04CF9A02001220421C005E6
:105C1800FCF752FE0123284A137089E732888A422A
:105C28000BD2B84205D00300318014E762463280B7
:105C38001EE7134B214A1A6022E7114A13601FE737
:105C480000780008FA020020FFFF00000278000830
:105C58000E0600200801002004780008F405002042
:105C680006780008F205002008780008FC050020E6
:105C7800FDFF00000070000808060020E07700081B
:105C8800100000200C020020F0040020FC0200207C
:105C98003800002088130000F80000200C000020C5
:105CA800C002002094060020AC060020000400502A
:105CB800000600201006002016000020D8770008F3
:105CC80010B525220024FA211B4B89005C609C60DA
:105CD8005C701C701C615C615C731C73DC611C6211
:105CE8005C761C769C62DC629C54013A9C540D32B2
:105CF8005C639C639C54013A9C540D321C645C6444
:105D08009C54013A9C540D4B1868FAF7F5F9802316
:105D180001385B0498420DD2C021094A0906506037
:105D28000848036A1B021B0A0B430362072394609B
:105D3800136010BDFEE7C046B80600200000002032
:105D480010E000E000ED00E0444B1A68002A05D09E
:105D58001A68013A1A60002A00D17AE0404B5A6862
:105D6800002A04D05A68013A5A60002A68D01A6991
:105D7800002A04D01A69013A1A61002A58D0DA694F
:105D8800002A04D0DA69013ADA61002A48D09A6A0E
:105D9800002A04D09A6A013A9A62002A36D05A6BCD
:105DA800002A04D05A6B013A5A63002A24D01A6C8C
:105DB800002A04D01A6C013A1A64002A12D0294B1E
:105DC8001A6801321A601968274A914201D10022E3
:105DD8001A60264A13780133DBB2092B00D9002355
:105DE8001370704701213D329954013A9A5C012A97
:105DF800E5D15A6C1A64E2E7012131329954013A2B
:105E08009A5C012AD3D19A6B5A63D0E701212532D3
:105E18009954013A9A5C012AC1D1DA6A9A62BEE7BA
:105E280001325A761A7E012AB1D11A6ADA61AEE7CE
:105E380001325A731A7B012AA1D15A691A619EE765
:105E480001325A701A78012A00D090E79A685A608D
:105E58008DE7074B01321A7080E7C046040700201F
:105E6800B8060020B0060020FFFFFF7FB406002020
:105E78000007002030B505280FD8012585F31088C4
:105E880000224300054C18188000231859609960B7
:105E98005A70255482F3108830BDFEE7B8060020FA
:105EA80005280ED8012383F310884300181800230F
:105EB800044A800011184B604B70135483F3108808
:105EC8007047FEE7B8060020052808D843001818D0
:105ED800054B80001B185A78D0B2012A01D0002047
:105EE800704700225A70FBE7B806002000280ED041
:105EF80001280DD0012383F31088064B064A186049
:105F08000023137083F310881378012BFCD170479A
:105F18000130EFE704070020000700200C4B70B5A4
:105F28000C4906001868FAF7E7F800210A4C704394
:105F38006568A268A3689A42FCD089189A4200D87A
:105F48004919C91A884201D91A00F3E770BDC04639
:105F58000000002040420F0010E000E070B500266D
:105F68000C4D0D4C641BA410A64209D1002600F06C
:105F78002BF80A4D0A4C641BA410A64205D170BD2B
:105F8800B300EB5898470136EEE7B300EB58984753
:105F98000136F2E71C6100081C6100081C6100085A
:105FA80020610008002310B59A4200D110BDCC5CD6
:105FB800C4540133F8E703008218934200D17047B4
:105FC80019700133F9E70000F8B5C046F8BC08BC01
:105FD8009E467047F8B5C046F8BC08BC9E46704758
:105FE800C004000890040008900400088E0400080B
:105FF8009404000894040008DC0500088E040008D6
:1060080094040008DC050008940400088E040008C5
:106018008805000888050008880500081806000893
:106028000000000000000000000000000000000068
:106038000000000000000000000000000000000058
:10604800010000000200000003000000040000003E
:10605800060000000700000008000000090000001A
:106068000000000000000000000000000000000028
:10607800010000000200000003000000040000000E
:1060880052360008E2350008E2350008E23500081B
:10609800B0360008E2350008E2350008E2350008AD
:1060A80016370008E2350008E2350008E235000836
:1060B80076370008E2350008E2350008E2350008C6
:1060C800D6370008E2350008E2350008E235000856
:1060D800EC35000804020800010002000400060074
:1060E80008000A000C001000200040008000000199
:1060F800080402040801010101010103070100006D
:106108004443452D323330322D56352E305F4841C9
:046118004C00000037
:04611C00E100000896
:04612000B9000008BA
:106124000024F4000100000004000000010000004D
:086134000070000846000101A3
:0400000508001401DA
:00000001FF
